:10000E004150545832410057494445312000574918
:05001E00444532200002
:102C8A0025E0FF900297E02402F582E43401F583FF
:102C9A0022EFF0900297E004F022EFF0900296E023
:102CAA0004F0A3E004F0227B017A01790290018307
:102CBA00E0FD227C007D0A120303ED2430229002FB
:052CCA009BE025E02263
:102BFA00E4F5AF120C29122CB1122753122CB11280
:102C0A00224E7FC01233EEE4FF1233EEE4900295B7
:102C1A00F0900183E0FF900295E0FEC39F50137489
:102C2A00022E122C93E0FF1233EE900295E004F08C
:0A2C3A0080DF7FC01233EE0233A7E3
:100C2900E4900297F0900296F0900296E090000E00
:100C3900936008122C8A122CA480EE122C8D7460F9
:100C4900122C9CE4A3F0A3F0A37408F0120F2DEF6B
:100C59006020120F2DEF122C8AEFF090029AE00417
:100C6900F07006900299E004F0122C9DA3E004F0C4
:100C790080DA900298E0C394065028E4900296F036
:100C8900900298E0FFC374069FFF900296E0C39F0D
:100C99005011A3122C907440122C9C900296E004DF
:100CA900F080DD7F0F7E0012324490029BEFF07FCF
:100CB900107E00123244EF24FE602804706D122C5D
:100CC900C844E0122C8C122C9BE4900296F09002FE
:100CD90096E0900015936008122C8A122CA480EEDD
:100CE900020D2D122CC844E0122C8C122C9BE4907E
:100CF9000296F0900296E0900015936008122C8AF3
:100D0900122CA480EE122C8D7462122C9CE4900299
:100D190096F0900296E090001C936008122C8A12BB
:100D29002CA480EE122C8D74638009122CC84461A6
:100D3900122C8CEF122C9C122C8D7403122C9C12E9
:100D49002C9074F0122C9C7F117E00123244122CCC
:100D59008D122C9BE4900296F0900296E02418F5EF
:100D690082E43403F583E0FF6008122C8D122CA471
:100D790080E77F127E00123244122C8D122C9BE4E4
:100D8900900296F0900296E0240EF582E43403F581
:100D990083E0FF6008122C8D122CA480E77F137E5C
:100DA90000123244122C8D122C9B9002FFE0FAA300
:100DB900E0FB7C007D64FFAE02120303EF243012D6
:100DC9002C8C122C9B7C007D0AAF03AE021203030C
:100DD900122CBDFF122C90122C9B9002FFE0FEA357
:100DE900E0FF122CBD122C8C122C9B122C90742F0C
:100DF900122C9C90030AE0FF75F064842430FE12E3
:100E09002C8DEE122C9CEF75F00A8475F00A84E59E
:100E1900F02430FF122C90122C9B90030AE075F0FD
:100E29000A84E5F02430122C8C122C9B122C90741D
:100E39002F122C9C122C907441122C9C122C907401
:100E49003D122C9CE4900296F0900296E0FFC39428
:100E590006501974032FF582E43403F583E0122C4C
:100E69008C122C9B900296E004F080DD900299E4AC
:100E7900F0A37440F0120F39EF601B120F39122CD6
:100E89008DEFF090029AE004F07006900299E00468
:100E9900F0122C9D80DF122C8D7420122C9C122DA7
:100EA90056E4900296F0900296E02432F582E434FA
:100EB90003F583E0FF6008122C8D122CA480E71241
:100EC9001455EF64017026122C8D7420122C9CE4A9
:100ED900900296F0900296E02428F582E43403F516
:100EE90083E0FF6008122C8D122CA480E7120F45B5
:100EF900300826122C8D7420122C9CE4900296F056
:100F0900900296E024D6F582E43402F583E0FF608E
:100F190008122C8D122CA480E7900297E09001838F
:030F2900F07F0155
:100F2C0022900299E0FEA3E0FF1232442290029933
:090F3C00E0FEA3E0FF12324422A2
:102BAD00E0FAA3E0FBFFAE02120303EF2430FF9027
:102BBD00029FE02428F582E43403F583EFF09002C0
:102BCD009FE004F0227C00AF03AE021203037C00F1
:102BDD007D0A120303ED22E02428F582E43403F587
:0D2BED008322E0FAA3E0FB7C007D0AFF22BA
:1014550012301CEF7002FF227FCC1200267F44124F
:10146500002630A0FD12301CEF7002FF227FCC1247
:1014750000267FBE1200261230E0900330E4F0A370
:10148500EFF01230E090032EE4F0A3EFF0E49002C9
:101495009FF090029FE0FFC39406500C74282F1212
:1014A5002BE7E4122BCA80EA90032EA3E0FF30E776
:1014B5001DD20BFE900331E02400FF900330E03E87
:1014C500FEEFF4FFEEF4FEEF2401FDE48012C20B03
:1014D50090032FE0FE900331E02400FD900330E0FF
:1014E5003EFCE41201F1E4FBFA7920783F12004654
:1014F50012022A9002A0EEF0A3EFF0E490029FF012
:10150500300B08122BE4742D122BCAC39002A1E0F4
:1015150094649002A0E09400500C122BEFAE0212DE
:101525000303EF02158EC39002A1E094E89002A098
:10153500E09403502C7C007D64122BAD7D0A122BA8
:10154500D22430FF122BBF122BE4742E122BCAA308
:10155500E0FEA3E0FF122BDB2430FF90029F021573
:10156500A8C39002A1E094109002A0E094275041F6
:101575007C037DE8122BAD7D64122BD22430FF1243
:101585002BBFA3122BEF122BD6122BB9122BE474FF
:101595002E122BCA7C007D0AAF03AE02120303EDA7
:1015A5002430FF122BBF122BE47443122BCA7F0188
:0315B500227F0092
:0115B8002210
:0731F900123200D2A07F0199
:10320000AE071FEE600D000000000000000000008F
:043210000080ED222B
:10301C00D2D7C2A07FF01232007FF0123200D2A0C1
:10302C007F3C123200A2A07FF01232007FB4123229
:0A303C000020D7037F01227F00224D
:1030E000E4FDFCEDC313FDC2A07F011231F930A055
:1030F00004ED4480FD7F3C1232000CECB408E4AFD8
:0131000005C9
:0131010022AB
:02002600AD0724
:10002800E4FCC2A07F01123200EDC313FD92A07F51
:090038003C1231F90CECB408E9AA
:01004100229C
:101F2400EF2430F09002CBE0FCA3E0FDA3E0FEA39D
:101F3400E022FFEE3395E0FDFCE0F8A3E0F9A3E036
:101F4400FAA3E022FFE4FAF9F8122CCFAC00AD01B9
:101F5400AE02AF039002CB0204E4F00B74D62BF56F
:101F640082E43402F58322A804A905AA06AB07E09B
:101F7400FEA3E0FFEE3395E0FDFC222FFFEA3EFED8
:101F8400E93DFDE83CFC2212036E78101204BD907A
:101F940002AB1204E49002AB221204BD9002A70229
:101FA40004E4EF2402FFE43EFEE43DFDE43C22F8B9
:101FB400E0FEA3E0FFE4FCFD12036E780F22FF12A3
:0F1FC4002CCFEF243022FB12036E780C0204BDE9
:1021B500121F587BA07A8679017800121F28FF121A
:1021C5002CCF9002E5121F24FF7BA07A8679017837
:1021D50000121F4DE47B107A27F9F8121F28FF1211
:1021E5002CCF9002D0121F24FFE47B107A27121FF8
:1021F5004BE47BE87A03F9F8121F28121FC29002FC
:10220500EF121F27FFE47BE87A03121F4BE47B6480
:10221500FAF9F8121F28121FC29002F0121F277B2D
:1022250064121F48E47B0AFAF9F8121F28121FC22C
:102235009002CF121F277B0A121F489002CBA3A33F
:09224500A3E024309002D1F02244
:0D332B00E4FF9002CBE004F00FEFB46EF56C
:013338002272
:0E333900E4F5D875F9DCF5E9D2DE30DFFD22CF
:0F32D100D2A4D2A312332BC2A412332BC2A32236
:0C33B400C2A4D2A312332BD2A402332BEC
:0E334700A20B92A4D2A312332BC2A302332BEB
:10325B00D2A312332BA2A430A404C2088002D2083A
:06326B00C2A312332B2266
:0231A500AE0773
:1031A700E4FDEE25E0FE92A4D2A312332BC2A312B4
:0A31B700332B0DEDB408EB02325B80
:10312400E4FED2A4FDEE25E0FED2A312332BA2A42A
:10313400E4334EFEC2A312332B0DEDB408E7AF0601
:013144002268
:022E0B00AC0712
:102E0D001232D17FEE1231A5AF041231A51232D19B
:102E1D007FEF1231A5123124AC07C20B12334712CA
:102E2D003124AD07D20B1233471233B4123339AFFD
:052E3D0004EFFEEDFFB3
:012E4200226D
:103145001232D17FEE1231A57FF41231A57F2E12F6
:1031550031A51233B41233397FF6122E0B121F78B4
:013165002247
:103046007F007E007D007C001232D17FEE1231A51A
:103056007FF41231A57F341231A51233B4123339FD
:083066007FF6122E0BE4FDFCC5
:01306E00223F
:1022E6007FAA122E0B9002F3EEF0A3EFF07FAC1252
:1022F6002E0B9002F5EEF0A3EFF07FAE122E0B90B0
:1023060002F7EEF0A3EFF07FB0122E0B9002F9EE7B
:10231600F0A3EFF07FB2122E0B9002FBEEF0A3EFCC
:10232600F07FB4122E0B9002FDEEF0A3EFF07FB615
:10233600122E0B9002D2EEF0A3EFF07FB8122E0B06
:102346009002D4EEF0A3EFF07FBA122E0B9002E6C5
:10235600EEF0A3EFF07FBC122E0B9002E8EEF0A396
:10236600EFF07FBE122E0B9002EAEEF0A3EFF02202
:100F450012314590029F1204E41230469002A3121A
:100F550004E49002FDE0FEA3E0FBAA0690029F12C6
:100F65001F2BC39BFBEE9AFAED9400F9EC940090CD
:100F750002FB121FB3121F9D9002E8121F73780B1C
:100F85001204D1C004C005C006C007A3E0FEA3E05B
:100F95009002A7121F362FFBEA3EFAE93DF9E83C1D
:100FA500F8D007D006D005D004122CCF121F93120B
:100FB5001F2BFF9002A7121F3D121F7F9002AF1239
:100FC50004E49002AF121F2B2408121FA9FC780419
:100FD5001204BD1221B59002F0E09002E0F09002FB
:100FE500CFE09002E4F09002D1E09002ECF09002A4
:100FF500AF121F2B2460FFEE34F0FEED34FFFDEC45
:1010050034FFFCA31204E49002B3121F2BFFA804C3
:10101500A905AA06121FCA9002D4121F6B12036EED
:10102500780B121F9D9002F5E0FEA3E09002B3122B
:101035001F36FB12036E780B121F90121F2BFF90A9
:1010450002A7121F3D121F7F9002B71204E49002FF
:10105500F3121F73E47B04FAF9F812036E9002B7DA
:10106500121F3D121F7F121FA6FCE47B04FAF9F83C
:10107500122CCF9002BB1204E49002F7121F73905A
:1010850002B3121F3DFB12036E780D121F9D9002D5
:10109500B3121F2BFF9002B3121F3D121FCA9002FD
:1010A500D2121F6B121F8B121F2BFF9002A7121F4C
:1010B5003D121F7F121FA6FC78021204BD9002B7D5
:1010C5001204E49002B7121F2B2400FFEE348012A5
:1010D5001FACAB07AA06A9059002F9121FB31204AB
:1010E500AA9002C31204E49002A3121F2BFFC004AE
:1010F500C005C006C0079002BB121F2BFBAA06A99C
:1011050005A804D007D006D005D004C3EF9BFFEE99
:101115009AFEED99FDEC98FCE47B507AC3F9F81240
:10112500036E9002C71204E4E4FFFEFD7C8090028A
:10113500C7121F3DFBC3120499501EE47F02FEFD3A
:10114500FC9002C7E0F8A3A3A3E012036E9002C3CC
:10115500121F3DFB1203F980189002C3121F3DFBBD
:10116500A3121F2BFF1203F9E47B02FAF9F812030D
:101175006E9002BF1204E49002BF121F2BFF780885
:101185001204BDC004C005C006C0079002BF121FEF
:101195002BFF78081204BDD003D002D001D0001275
:1011A500036E121FA0E47FDE7E0BFDFC9002A712EA
:1011B5001F3DFB12036E7810121F9D7F437EE37D5A
:1011C500FF7CFF9002BF121F3DFB121F8B121F2BCE
:1011D500FF9002A7121F3D121F7FEF24CFFFEE34B1
:1011E5000E121FACFC78041204BD9002BF121F3D05
:1011F500121F7F1221B59002E5E0FF9002EEF090FC
:1012050002D0E0FE9002F2F09002EFE0FD9002E1E4
:10121500F09002F0E0FC9002EDF09002CFE0F99042
:1012250002F1F0E4FB24D6121F63EF121F5EEE12EB
:101235001F5EED121F5EEC121F5E742E121F5EE91B
:0F124500121F5E7470F074D62407121F63E4F05A
:011254002277
:10259B001203F9EB2430FF9002A3E02432F582E41E
:1025AB003403F583EFF09002A3E004F0E02432F55E
:1025BB0082E43403F583227F07122E43E4FCFD12E1
:1025CB0001ECE4FBFA79407840120046E4FBFA791F
:1025DB0080784412014FE4FBFA227B0AFAF9F89057
:1025EB00029FE0FCA3E0FDA3E0FEA3E0FF227948FD
:0F25FB00784312004602022A900293E0940122D4
:0D338D00439180439280439D8075BCA02237
:102E4300E4F5BDF5BEE5BC54E044084FF5BC000015
:102E530000007DFAE5BC30E41753BCEFAFBDEF755E
:102E6300F004A4FFACBEEC7A002FFFEA35F0FE229B
:062E7300DDE27E037FFF9B
:012E79002236
:102D56001225C279A078411225FD90029F1204E443
:102D6600E49002A3F01225E51203F9E47B0AFAF9CE
:102D7600F812259B742EF09002A3E004F0E41225CD
:102D8600E512259B74561225B0E4F09002A3E004E8
:012D9600F04C
:012D97002219
:1028EC001225C21225F9900293EEF0A3EFF0C394D7
:1028FC009AEE940140047F068042C3900294E094C7
:10290C007C12260340047F058032C3900294E0942D
:10291C005E12260340047F048022C3900294E0944C
:10292C004012260340047F038012C3900294E0946B
:0F293C003112260340047F0280027F011230BC5B
:01294B002269
:10267900E490029BF0A3F0A3F07F07122E43E4FC41
:10268900FD9002971204E49002971225EDE41225B9
:10269900CA1225F99002931204E4900293A3122519
:1026A900F290029CE02FF090029BE03EF090029D98
:1026B900E004F0E0C3940A40C090029BE0FEA3E06E
:1026C900FF7C007D0A12030390029BEEF0A3EFF05A
:0D26D900C39431EE940150037F01227F0075
:0126E60022D1
:1030BC00900295EFF0900295E0FF14F0EF6014C2CF
:1030CC00907F037E00123187D2907F037E001231F5
:0430DC008780E222E5
:10318700EF4E6019EF1FAC0670011E4C600FE4F59F
:0E319700D875F94CF5E9D2DE20DFE980FB2285
:1032C00041542B4E414D453531544E432D583241DA
:0132D00000FD
:0D339A00D2C2D280D290D282D283D28122C0
:1031C1001226E71233E4122EDF122826122A0412E5
:0C31D1002118122679BF01EBC20980E72B
:102EDF0020962D7F017E00123187209623B28430F9
:102EEF0084107F147E001231877BFF7A3279C012F3
:102EFF00329A3096FD7F017E001231873096F32291
:012F0F00229F
:102FC6002096277F017E0012318720961D7F0112F1
:102FD60015B9C2C2C290C282C2813096FD7F017EFF
:0B2FE600001231873096F375C72022DF
:030003000229AA25
:1029AA00C0E0C0F0C083C082C0D075D000C000C0F3
:1029BA0001C002C003C004C005C006C00720B21F80
:1029CA007F017E0012318720B215B20930B2FD7F35
:1029DA00017E0012318730B2F330090375C720D067
:1029EA0007D006D005D004D003D002D001D000D041
:0A29FA00D0D082D083D0F0D0E032BC
:0A33E40020090612335575870222F6
:0E335500C294C284C2C0D2B6D2B712339A223A
:1026E700123355D209D2C01233FF75BBFFE4F591FF
:1026F700759220F5B375B40143B70243B80243B7E7
:1027070010C2C2C280C290C282C283C2817F0AFE47
:1027170012318712339A12322C122FC612338D12AE
:1027270032E01234061222E61214551214551230F2
:102737006FC28CE490033CF0C28CC28D758C4CF553
:0C2747008AD28CD2A8D2A9D2AF0228EC12
:03000B00022AB412
:102AB400C0E0C0F0C083C082C0D075D000C000C0E8
:102AC40001C002C003C004C005C006C007C28CC256
:102AD4008D758C4C758A00D28C90033CE004F0E038
:102AE400D394144005E4F0122496D007D006D00500
:102AF400D004D003D002D001D000D0D0D082D08373
:052B0400D0F0D0E0322A
:1016F100504F5745523A200020202054454D503A32
:101701002000202D2D2D2D2D200020202050726510
:1017110073737572653A2000200D0A0D0A00415459
:101721002B48454C503D310D0A0041542B44454D49
:101731004F3D310D0A0041542B43414C4C3D000DAE
:101741000A0041542B535349443D0041542B444911
:1017510047493D0041542B54494D453D0041542BCF
:10176100424541434F4E3D000D0A0D0A002A2A2AE7
:101771002041505253203531547261636B205832ED
:101781004128424C41434B424F5829203230313499
:10179100313231352042483454445620202A2A2AF5
:1017A100200D0A004E4F43414C4C00333133342E4F
:1017B10035354E000031323032302E36364500415B
:1017C100505253203531547261636B20583241209D
:1017D10021000000000000000000000000312C3456
:1017E10033382E353030302C3433382E35303030DC
:1017F1002C302C332C300000000000312C313434DB
:101801002E363430302C3134342E363430302C30C6
:091811002C332C302C30000000B7
:10288B0090029CE0FEA3E0FFE4FD1231DDE004F0DA
:10289B002290029BA3E02400F582E43400F583220E
:1028AB0090029BE0FEA3E0FF2290029CE004F0224A
:1028BB0090029CE0FEA3E0FF2290029BE004F0223A
:1028CB0075C65A75C6A52290029CE4F0A322ECF5BE
:1028DB00C3AF058FC422F0A3EFF0C3940AEE9400AC
:0128EB0022CA
:10089600E490029DF0A3F090029BF0A3F090029DDD
:1008A600E0FEA3E0FF12324412289CEFF090029E75
:1008B600E004F0700690029DE004F090029CE004D3
:1008C600F070031228C4C390029BE0940140CE7BD3
:1008D600FF7A17796E122F6E122D567BFF7A1679D4
:1008E600F1122F6E7B017A037932122F6E7BFF7A1B
:1008F6001679F9122F6E121455BF01087B017A037F
:10090600792880067BFF7A177903122F6E7BFF7A90
:1009160017790B122F6E120F453008087B017A02E9
:1009260079D680067BFF7A177903122F6E7BFF7AC2
:10093600177919122F6E7BFF7A17791F122F6E7B8C
:10094600FF7A17792B122F6E7BFF7A177937122FC2
:100956006E90029BE4F0A37408F012289CE0FF60FE
:100966000A120BF170F41228C480EF120BD47A1716
:100976007943122F6E90000FE0FF7E0090029BEEEF
:100986001228E11228AB7C007D0A5002800A120B65
:10099600A61228AB7C007D0A120C07120BD47A171C
:1009A600794C122F6E900005120BC7900006120BA1
:1009B600C7900007120C12900004E02430FF123397
:1009C600EE120BFB7A177955122F6E900000E0FE9F
:1009D600A3E07C002400FFEC3EFE90029B1228E17F
:1009E600500B90029BA3E02430FF1233EE1228AB8B
:1009F600D39409EE940040047D0180027D00C3EF8C
:100A06009464EE940050047F0180027F00EF5D60E5
:100A160003120B721228ABD39463EE940040047D4C
:100A26000180027D00C3EF94E8EE940350047F0139
:100A360080027F00EF5D600D1228AB7C007D6412A2
:100A46000BA6120B721228ABD394E7EE9403400464
:100A56007D0180027D00C3EF9410EE942750047F41
:100A66000180027F00EF5D6006120B12120BB812B6
:100A760028ABD3940FEE942740147C277D101203E5
:100A860003120BB8120B127C007D0A120C07120B14
:100A9600FB7A17795E122F6E900010120C129000DE
:100AA60011120BE07420F012289CE0FF600A120B72
:100AB600F170F41228C480EF7F2C1233EE900012EE
:100AC600120BE07430F012289CE0FF600A120C1F33
:100AD60070F41228C480EF7F2C1233EE900013E0DE
:100AE600FF1233EE7F2C1233EE90029BE4F0A374D8
:100AF60040F012289CE0FF600A120C1F70F41228C6
:0C0B0600C480EF7BFF7A177969022F6E24
:100B120090029BE0FEA3E0FF7C037DE81203037CCE
:100B2200007D0A120303ED2430FF1233EE90029B84
:100B3200E0FEA3E0FF7C007D641203037C007D0ADB
:100B4200120303ED2430FF1233EE90029BE0FEA36A
:100B5200E0FF7C007D0A1203037C007D0A1203037E
:100B6200ED2430FF1233EE90029BE0FEA3E0FF2261
:100B720090029BE0FEA3E0FF7C007D0A1203037C4F
:100B8200007D0A120303ED2430FF1233EE90029B24
:100B9200E0FEA3E0FF7C007D0A120303ED2430FF98
:100BA2001233EE221203037C007D0A120303ED24AA
:100BB20030FF1233EE227C007D0A120303ED243053
:100BC200FF1233EE22E02430FF1233EE7F2C123379
:100BD200EE227BFF7A177940122F6E7BFF22E0FF15
:100BE2001233EE7F2C1233EE90029BE4F0A322121A
:100BF20033EE90029CE004F0227BFF7A17794012D8
:100C02002F6E7BFF22120303ED2430FF1233EE22FC
:100C1200E02430FF1233EE7F2C1233EE221233EE39
:070C220090029CE004F022A7
:1032140090029EEFF07F007E0212328790029EE0C1
:08322400FD7F007E020231DD96
:102B5C00E4FFFE123287E490029DF0A3F090029BFA
:102B6C00F0A3F090029BE0FCA3E0FDC3EC940150B9
:102B7C002FA3E0FEA3E0FF74002D1228A3E0FD12AA
:102B8C0031DD90029EE004F0700690029DE004F0AE
:102B9C0090029CE004F070CB90029BE004F080C3A8
:012BAC002206
:10322C007F1F7E00123244EF64997F0160091215F2
:08323C00B975C7207F002222B2
:0E336300E4F5C7F5C5F5C675C3FF75C4FF22B6
:04324400AD07AC0620
:1032480075C78275C5011228D91228CB00AFC212E2
:023258003363DE
:01325A002251
:10328700AD07AC061228D975C78275C5031228CBBE
:033297000233639C
:102F4100AD07AC0675C78275C5021228D91202AB4E
:102F5100F5C21228CB000DBD00010C740129F9E462
:0D2F61003AFA9002A3E014F070E00233632E
:1031DD00AB07AA0675C78275C502EAF5C3AF038FA3
:0C31ED00C4AF058FC21228CB0002336370
:0515B90090029BEFF021
:1015BE00E4FFFE1232877BFF7A1779A59002A3749F
:1015CE0007F07F08122F417D097F0F1231DD7D015B
:1015DE007F041231DD1D7F051231DD7F061231DDF4
:1015EE000D7F071231DD0DE4FF1231DD7D587F01D5
:1015FE001231DD7D017F101231DD7D217F1112311F
:10160E00DD7D2F7F121231DD7D3E7F131231DD1213
:10161E0028D27420F0E4FCEC9017AC93FD600E120F
:10162E0028BB12289570031228B40C80EA12288B5E
:10163E0070031228B41228D27430F0E4FCEC901728
:10164E00B693FD600E1228BB12289570031228B4B3
:10165E000C80EA12288B70031228B41228D2744020
:10166E00F0E4FCEC9017C093FD600E1228BB12281C
:10167E009570031228B40C80EA12288B700312287E
:10168E00B490029BE07028A3F0A37480F0E4FCEC0D
:10169E009017DE93FD600E1228BB12289570031270
:1016AE0028B40C80EA12288B70031228B4802612FC
:1016BE0028D27480F0E4FCEC9017FC93FD600E12BF
:1016CE0028BB12289570031228B40C80EA12288BBE
:1016DE0070031228B47D997F1F7E001231DDE4FF66
:0316EE00023214B1
:101DC4000D0A2020B2BBC8CFCAB6C4E3CAE4C8EB2C
:101DD400B5C4D6B8C1EEA3ACBFC9C4DCC3BBBCD3C5
:101DE400BBBBD0D0C5B6A3A120A3BAA3A920200D04
:101DF4000A0D0A0041542B48454C503D31004154D2
:101E04002B44454D4F3D310041542B54494D453DE4
:101E14000041542B43414C4C3D0041542B535349F6
:101E2400443D0041542B424541434F4E3D004154F3
:101E34002B444947493D000D0A202D3E20C9E8D6D0
:101E4400C3B3C9B9A620202120200D0A000D0A2001
:101E54002D3E20D6B8C1EEB4EDCEF3A3A1BFC9C4C4
:101E6400DCC8B1C9D9BBD8B3B5A3A120200D0A00E1
:101D0500900294E02400F582E43400F583E4F09039
:101D15000293E004F0E02407F582E43402F583E061
:101D250022900210E024D0FFE434FFFE7C00120272
:101D3500F1AA06AB0790020FE024D0FFE434FFFEC2
:101D450022900294E02400F582E43400F5832274A5
:101D550008900293F0E4900297F0A3F022EFF09040
:101D65000293E004F022900298E004F0229002979A
:101D7500E004F0227D0A1202F1EF2BFFEE3AFE227B
:101D8500900287E0FF2406F582E43402F583E02221
:101D95001202F1EF2BFBEE3AFA22900294F0900238
:101DA50093227B017A017902900183E0FD22900262
:0F1DB50097E0FEA3E0FFEE2290020FE024D02281
:030023000227BFF2
:0D27BF00C0E0C083C082C0D075D000C0074C
:1027CC00309906C299D2078046309843300604C22D
:1027DC0098803C7F80900207E4F0A3DFFC7F0075BB
:1027EC00D80075F94C75E900D2DE20980C30DFFA70
:1027FC00900287EFF0D2068016C29874072FF582EC
:0F280C00E43402F583E599F00FEFD3947F40D0C9
:0B281B00D007D0D0D082D083D0E032B4
:102118002006030221B4900207E064C0704EA3E0D9
:10212800704A121D8564C07043EFD39411403DE49A
:10213800900183F07F02900287E014FEEFC39E5067
:102148001C74072F121D1DFE74002FF582E4340144
:10215800F583EEF0900183E004F00F80D9121DA7FB
:10216800122753121DA712224EC20622121D85B431
:102178000A047E0180027E0074052FF582E4340291
:10218800F583E0B40D047F0180027F00EF5E6008F4
:10219800E4F5AF1204F0800FE4F5AF1208967BFF68
:0C21A8007A1D79C4122F6EC2061233A7F4
:0121B4002208
:1004F000E4900299F0A3F0121D5B900299E0FEA334
:10050000E0FF123244900297A3121D49EFF09002CF
:100510009AE004F07006900299E004F0121D6B70EE
:1005200003121D72C3900297E0940140CD7BFF7AC5
:100530001D79F8123166BF01030208967BFF7A1E0F
:100540007902123166BF010BE4FF1215B91233C0F4
:1005500075C7207A1E790C120873600302063412E4
:100560001D54900293121D1A640D600D121D641229
:100570001D6B70EE121D7280E9121DB3600302063E
:100580001BEF24FE602114602A14603714604E248F
:1005900004600302061B121DBDFEE434FF900295A9
:1005A000F0A3CEF0020622121D3A7C007D0A120250
:1005B000F180277D0A121D267D64121D7B90021199
:1005C0000206067D64121D267C037DE8121D9590AF
:1005D0000211121D3D7C00121D79A380299002108A
:1005E000121D3D7C037DE8121D337C277D10121DFA
:1005F00095900211121D3D7C007D64121D95A31281
:100600001D3D121D79A3E024D0FDEC34FFCD2FFF5A
:10061000ED3E900295F0A3EFF08007E4900295F094
:10062000A3F0900295E0FCA3E0FDEC900000F0A3A5
:10063000ED12088E7A1E79151208737074121D540B
:10064000900293121D1A640D600D121D64121D6B31
:1006500070EE121D7280E9D3900298E09406900229
:1006600097E0940040031233CC900297E07002A30D
:10067000E070031233CC7408121D9FF0900298E0D2
:100680002408FF900297E03400FE900293E0FDC33F
:100690009FE49E501674072D121D1DFF121D46EF7C
:1006A000F0900294E004121D6380D1121D461208DE
:1006B0007C7A1E791E120885704B121D549002938D
:1006C000121D1A640D600D121D64121D6B70EE1266
:1006D0001D7280E9121DB37020EF24FE60080470C3
:1006E00018121DBD800D121DBD75F00AA4FFA3E0F8
:1006F00024D02F90000FF0800690000F740AF012A3
:100700002B5C1233C07A1E7927120885600302071A
:10071000F0740A121D56900293121D1AFF640D60A8
:1007200011EFB42C08121D6B7003121D72121D64A0
:1007300080E4900297E07004A3E06406600302087E
:1007400029900293740A121D1924D0900010121DD2
:1007500013642C60031233CC121D14900011121D6F
:1007600013642C60031233CC7420121D9F801290EE
:100770000293121D1AFF642C600C121D46121D629A
:10078000A3E004F080E9121D05900012121D13640D
:100790002C60031233CC9002947430F0900293805A
:1007A00012900293121D1AFF642C600C121D461247
:1007B0001D62A3E004F080E9121D05900013121DD4
:1007C00013642C60031233CC9002947440F09002B6
:1007D000938012900293121D1AFF640D600C121D7B
:1007E00046121D62A3E004F080E9121D4612087C47
:1007F0007BFF7A1E7932123166EF64017074121D2C
:1008000054900293121D1AFF640D6011EFB42C086E
:10081000121D6B7003121D72121D6480E49002970A
:10082000E07004A3E0640360030233CC900293748D
:1008300008121D1924D0900005121D13642C6003AA
:100840001233CC121D1424D0900006121D13642CF8
:1008500060031233CC121D1424D0900007121D1314
:10086000642C60031233CC121D1424D090000412A7
:02087000088EF0
:10087200227BFF123166EF640122E4F0122B5C123C
:1008820033C0227BFF123166EF640122F0122B5C2F
:040892001233C0223B
:0C33C0001208967BFF7A1E793B022F6EEC
:0C33CC001208967BFF7A1E7951022F6ECA
:10316600E4FF1202ABFE601674072F121D1D6E607F
:10317600037F00220F740129F9E43AFA80E47F0103
:013186002226
:0F32E000759850759CFD758E11758911023271AC
:10327100C2ACC206E4900287F07F80900207E4F0BE
:05328100A3DFFCD2AC4C
:013286002225
:102F6E0090029FEBF0A3EAF0A3E9F090029FE0FB42
:102F7E00A3E0FAA3E0F91202ABFF600F1233EE905A
:0C2F8E0002A0E475F00112035880E0225C
:0A33EE00C2078F993007FDC20722C5
:101939000F90028BE0FBA3E0FAA3E0F98F82758395
:10194900000202C4FD74182EF582E43403F583ED18
:10195900F00E0F2290028BE0FBA3E0FAA3E0F9223C
:1019690090028CE0900304F090028DE0900305F062
:1019790090028EE0900306F090028FE0900307F04A
:101989009002902290028DE0900304F090028EE084
:10199900900305F090028FE0900306F0900290E02A
:1019A900900307F090029122FD740E2EF582E43423
:1019B900032290028CE0900305F090028DE09003E1
:1019C90006F090028EE0900307F090028F229002B9
:1019D9008BE0248CF582E43402F583EEF090028BDF
:1019E900E004F00F22EBF0A3EAF0A3E9F0E422907F
:1019F900028CE0900306F090028DE0900307F090CE
:101A0900028E22F09002FFE0FFA3E0900322CFF0C4
:101A1900A3EFF07F012290028EE024D022748E2D54
:101A2900F582E43402F583EFF00C0D22C294C20072
:101A3900D28022FFE434FFFE7C007D0A0202F1908D
:0B1A4900028CE0900307F090028D2259
:102EAD0020932E7F017E00123187209324900325DD
:102EBD00E004F0E0D394044002E4F0900325E0FF39
:102ECD001232143093FD7F017E001231873093F35F
:022EDD002222AF
:102A0400122EAD900325E024FE601514603314608B
:102A140033240370339003247401F0D294022F9A68
:102A2400900324E064026003122F109003247402C4
:102A3400F0D294300222C20230001D122BFAC200DE
:102A440022022A5D121A3522E4900324F020940510
:092A54001233A7D294122FF122D3
:102F1000E4FFFE123244EF7F00FEC006C0070F7EC2
:102F200000123244EFFDD0E02DFFD0E03400FE90DF
:102F30000326F0A3EFF0900301EEF0A3EFF0C2023E
:012F4000226E
:102A5D00900324E0640360097403F0121A35122FF9
:102A6D0010300242C2021233A7D294E4900293F0C6
:102A7D00A3F02000287F147E00123187900294E08D
:102A8D0004F07006900293E004F0D3900294E09469
:102A9D002C900293E0940140D9121A3522122BFA90
:062AAD00121A35122F1071
:012AB3002200
:10249600900325E024FE60121460171460252403BF
:1024A6007029D281D282B2838027B281D282D2832E
:1024B600801FD283308206C282C2818014D282D229
:1024C60081800ED281B282D2838006D282D283D21A
:1024D60081900326E0FEA3E0FF4E601F900302E01A
:1024E60024FFF0900301E034FFF0E07002A3E070F7
:1024F6000A900301EEF0A3EFF0D20290030CE00481
:10250600F0700690030BE004F0D390030CE0940403
:0F25160090030BE094004006E4F0A3F0D2012202
:102FF1003091037F00227F017E00123187309103DF
:103001007F00223091FD7F017E001231873091F3E4
:0B301100300005122BFAC2007F0122E4
:102F9A0030000D122525BF0107122BFAC20080123C
:102FAA0030011830000C122C44BF0106122BFAC251
:0C2FBA000022E490030BF0A3F0C20122FF
:10306F00E4900322F0A3F090030DF0C2009003242C
:10307F00F0122F10E490030BF0A3F0FF7E02123238
:07308F0044900325EFF0223D
:031B5A009002886E
:101B5D001219EEFFFE90028812193DFD6009B42C9A
:101B6D00010E0FEEB409EE90028812193D642D702E
:101B7D00600F90028BF090028812193DFE642E606A
:101B8D00051219D780F07F069003037430F0A3DFA0
:101B9D00FC900303742DF090028BE024FE6013146F
:101BAD0060151460171460192404701A90028C02C9
:101BBD001BD6121A4880121219F8800D1219BB800B
:101BCD0008121969800312198DE0900308F0021CA8
:101BDD003EE490028BF090028812193DFE642E6057
:101BED00051219D780F07F069003037430F0A3DF40
:101BFD00FC90028BE024FE60131460161460181420
:101C0D00601A2404701B90028C021C39121A4802AF
:101C1D001C391219F880151219BB80101219698020
:101C2D000B90028CE0900303F012198DE0900308E5
:061C3D00F0E4900309F041
:011C4300227E
:032D1300900288A3
:102D16001219EEFFFE90028812193DFD6009B42CCF
:102D2600010E0FEEB402EE90028812193DB441195D
:102D36007B017A017985121E747B017A01798512ED
:0F2D46001A54C280D2007F0122B280C2007F00E7
:012D5500225B
:031E740090028B4E
:101E77001219EEFFFE12193A6009B42C010E0FEE8B
:101E8700B403F2E4FE12193AFD642E600512194EEE
:101E970080F390028B12196012194E12194512190C
:101EA7004D12194512194D12193A642C60030F800F
:101EB700F612193912194D74182EF582E43403F508
:101EC70083E4F012193A642C60030F80F60FE4FEE6
:101ED70012193AFD642E60081219B212195680F0D1
:101EE70090028B1219601219B21219561219451263
:101EF70019B11219561219451219B1121956121998
:101F07003A642C60030F80F61219391219B1F58360
:0C1F1700EDF00E1219B2F583E4F07F012A
:011F2300229B
:1025250090030AE07002FF22900322E0FEA3E0FF81
:102535009002FFE0FAA3E0FBD39FEA9E4008EB9FE1
:10254500FDEA9EFC80159002FFE0FEA3E0FFC3902C
:102555000323E09FFD900322E09EFCD3ED94B4ECB1
:102565009400401074689D900294F074019C900250
:1025750093F08008900293ECF0A3EDF0D3900294D1
:10258500E09419900293E094004008E490030D1242
:052595001A0C227F007A
:01259A00221E
:102C440090030AE0FE7002FF2290030DE004F0EE10
:102C5400C3940A500AE0940B400280227F00229021
:102C6400030AE0C39432500D90030DE09407400230
:102C7400800C7F002290030DE0D394054005E412FC
:062C84001A0C227F002261
:031A540090028B72
:101A57001219EEFCFD12195D8C821219476009B448
:101A67002C010D0CEDB407ED12195D8C821219478C
:101A7700B42C03E4804BE4FD12195D8C82121947E4
:101A8700FF642E6005121A2680EEED24FD60120415
:101A9700702C121A1F75F00AA4FFA3E024D02F8020
:101AA7002090028FE024D075F00AA4FF121A1F7548
:101AB700F064A42FFF900290E024D02F8003121A25
:101AC7001F90030AF012195D8C82121947642C606B
:101AD700030C80F10C12195D8C82121947B42C0883
:101AE700E49002FFF0A3F022E4FD12195D8C82124C
:101AF7001947FF642E6005121A2680EEED24FD605B
:101B07000C047040121A1F121A3CA3802390028FF4
:101B1700E024D0121A3CAA06AB07121A1FFFE434BE
:101B2700FFFE7D641202F1EF2BFFEE3AFE9002906A
:101B3700E024D0FDEC34FFCD2FFFED3E9002FFF007
:101B4700A3EFF022121A1FFEE434FF9002FFF0A366
:021B5700CEF0CE
:011B59002269
:0E337100244750524D43002447504747410027
:10310200A3F07B017A01798522900206E02485F5FD
:1031120082E43401F58322E0FBA3E0FAA3E0F902A2
:0231220002ABFE
:03004300021C4458
:101C4400C0E0C0F0C083C082C0D075D000C000C066
:101C540001C002C003C004C005C006C007E59A3035
:101C6400E106539AFD021CEAE59A30E079539AFEA4
:101C740012310BE59BF0900206E004F0900184E041
:101C840004F0E59B640A705312310BE4F0900206F1
:101C9400E004F0200A2190028B74FFF0A37433F067
:101CA4007471123102122DD2EF64017027123104C3
:101CB400122D13D20A801D90028B74FFF0A374338B
:101CC400F07478123102122DD2BF010812310412BD
:101CD4001B5AC20A900206E4F0800B900206E0D37D
:101CE400947E4002E4F0D007D006D005D004D0039F
:101CF400D002D001D000D0D0D082D083D0F0D0E0B8
:011D040032AC
:102DD200900288EBF0A3EAF0A3E9F090028B1231A3
:102DE20019FF60229002881231196F60037F00225E
:102DF200900289E475F00112035890028CE475F098
:092E02000112035880D57F012262
:06340600759A500233A785
:0D33A700E4F5AFC200900206F075AF012200
:0F32EF00E4F5D875F9FF75E9A0D2DE30DFFD22D6
:102E7A00E4FD7016C2B11232EF7E08EFC313FF925F
:102E8A00B11232EFDEF5D2B18015D2B11232EF7E35
:102E9A0008EFC313FFB392B11232EFDEF4C2B112DC
:022EAA0032EF05
:012EAC002203
:10329A001202ABFF600C122E7A740129F9E43AFA91
:0332AA0080EE2291
:10309600E4F5D875F9FDF5E9D2DE22C313F04480D4
:1030A600F0900182E004F022D2C2D280D290229027
:0630B6000100E0640322AA
:1028260020B561C2ACE4F5AF1230AE121FD39002F0
:1028360093EFF01232711233A7900293E0640170A5
:10284600431230AEC2C27FC01233EEE4FF1233EE43
:10285600E4900294F0900183E0FF900294E0FEC3BE
:102866009F501774022EF582E43401F583E0FF12BF
:1028760033EE900294E004F080DB7FC01233EED298
:04288600C21232AD9B
:01288A00222B
:0E224E00900297EBF0A3EAF0A3E9F0A3EDF005
:10225C00C2AC1230AEC290C2B6D2B7D295D2B3E4F1
:10226C00900182F090029BF01222DAE0C3944C4071
:10227C00F7E490029BF090029AE0FFA3E0C39F501A
:10228C0024900297E0FBA3E0FAA3E0F91202ABFF63
:10229C0012294C900298E475F00112035890029B9D
:1022AC00E004F080D190033BE0FF12294C90033AFC
:1022BC00E0FF12294CE490029BF01222DAE0C39466
:0E22CC000A40F7D2B6C2B7C295D29002327164
:0C22DA007F7E12294C90029BE004F02251
:101FD3001220791230B560037F0022900101E0B432
:101FE3007E0B12260A1230B560F17F0022E49002C4
:101FF30095F0900101E0FF647E602C900295E0244F
:1020030002F582E43401F583EFF0900295E004F0E9
:1020130012260A900295E0D3947840037F0022129F
:1020230030B560CE7F00227B017A01790290029560
:10203300E024FEFD122753900295E0FE2400F58272
:10204300E43401F583E0FF90033BE06F60037F001E
:102053002274012EF582E43401F583E0FF90033A04
:10206300E06F60037F0022900295E024FEF0E09091
:052073000183F07F0174
:012078002245
:10207900E4900100F01233F81233F8E4900101F012
:1020890030B40A30B5FA9001007401F02220B40A84
:1020990030B5FA9001007402F022A2B49204E490DF
:1020A9000182F0900296F012330D900101E0C31302
:1020B900F0900182E0B40616900296E004F0E0B4D4
:1020C900030C9001007403F0E4900182F022E49083
:1020D9000182F0C2052005CF12309620DF1C30B5F1
:1020E900079001007404F022A2B4300401B350EB4C
:1020F900A2B49204D205D2DF80E12005D890010173
:0E210900E01230A1E0B407CD9001007405F0A3
:0121170022A5
:10260A00E4900296F0900296E0C39408506012306B
:10261A009620DF2030B5079001007404F022A2B49E
:10262A00300401B3500AA2B49204D205D2DF80E189
:10263A00C20580DD200515900101E0FF1230A1E0FE
:10264A00B407079001007405F022801A12330D9026
:10265A000182E0B40504E4F080AB900101E0C31309
:0E266A00F0E4900182F0900296E004F0809778
:01267800223F
:05294C0090029CEFF079
:10295100BF7E04D2038002C203E490029DF0900284
:102961009CE054017004B2B380231230A720030409
:102971007F0180027F00900182E0B405047E018026
:10298100027E00EE5F600A1232FEB2B3E490018271
:10299100F090029CE0FFC313F01232FE90029DE022
:0829A10004F0E0C3940840B605
:0129A900220B
:0F32FE00E4F5D875F9FD75E908D2DE30DFFD2261
:0733F80012309630DFFD22C8
:0F330D00E4F5D875F9FE75E980D2DE30DFFD22D8
:0733FF00C295D2B6C2B7224D
:10125500000011892312329B462457AD653674BFB1
:101265008C489DC1AF5ABED3CA6CDBE5E97EF8F761
:10127500108101083393221A56A5472C75B7643E91
:101285009CC98D40BFDBAE52DAEDCB64F9FFE87641
:101295002102308B02101399672676AF443455BD71
:1012A500AD4ABCC38E589FD1EB6EFAE7C87CD9F521
:1012B5003183200A1291031877A7662E54B5453C51
:1012C500BDCBAC429ED98F50FBEFEA66D8FDC97401
:1012D5004204538D6116709F042015A9273236BB31
:1012E500CE4CDFC5ED5EFCD7886899E1AB7ABAF3E1
:1012F5005285430C7197601E14A1052837B3263A11
:10130500DECDCF44FDDFEC5698E98960BBFBAA72C0
:101315006306728F4014519D252234AB063017B9F0
:10132500EF4EFEC7CC5CDDD5A96AB8E38A789BF1A0
:101335007387620E5095411C35A3242A16B10738D0
:10134500FFCFEE46DCDDCD54B9EBA8629AF98B7080
:1013550084089581A71AB693C22CD3A5E13EF0B7B0
:10136500084019C92B523ADB4E645FED6D767CFF60
:1013750094898500B79BA612D2ADC324F1BFE03690
:1013850018C109483BD32A5A5EE54F6C7DF76C7E40
:10139500A50AB48386189791E32EF2A7C03CD1B570
:1013A500294238CB0A501BD96F667EEF4C745DFD20
:1013B500B58BA40296998710F3AFE226D0BDC13450
:1013C50039C3284A1AD10B587FE76E6E5CF54D7C00
:1013D500C60CD785E51EF497802891A1A33AB2B330
:1013E5004A445BCD695678DF0C601DE92F723EFBE0
:1013F500D68DC704F59FE41690A98120B3BBA23210
:101405005AC54B4C79D7685E1CE10D683FF32E7ABF
:10141500E70EF687C41CD595A12AB0A3823893B1EF
:101425006B467ACF485459DD2D623CEB0E701FF99F
:10143500F78FE606D49DC514B1ABA02292B98330CF
:101445007BC76A4E58D5495C3DE32C6A1EF10F787F
:05275300900297EDF07B
:1027580074FFA3F0A3F0900297E0D39400403F12D7
:1027680002ABFF900298A3E06F25E0FFE433FE740C
:10277800552FF58274123EF583E493FC740193FDA2
:10278800900298E0FFECFEED6FFFEEF0A3EFF09003
:102798000297E014F0740129F9E43AFA80B890023B
:1027A80098E0FEA3E0F4FFEEF4FCEF90033BF0AEFC
:0627B80004EE90033AF06C
:0127BE0022F8
:0E337F0057494445312000574944453220004B
:102B09001FEF25E0FF74022EF582E43401F583ED11
:102B190054E1F074022EF582E43401F58322749DA8
:102B29002FF582E43402F58322F0900298E004F054
:102B390022EE75F007A414F0AF067BFF227B017A21
:102B4900017902900183E0FD2290029BE4F0A374D5
:032B590008F0225F
:1032AD0090010FE020E00B122376EF640160031212
:0332BD00240622C2
:102376009002957403F07F057E00123244EF6401EB
:10238600707B900295E0FED3940840037F00229074
:102396000296122B3A7A33797F122D98EF640170E8
:1023A60043900296E0FE2402122B1FE0FD541EC34A
:1023B60013FF7002FF22122B09E04FF0EF700D9011
:1023C6000296E02402122B1FE04480F07F077E0075
:1023D600123244BF0108900295E0FF12181A123318
:1023E6001C7F0122900296E02402122B1FE030E0AF
:0F23F600037F0022900295E004F00223887F000D
:0124050022B4
:102406009002957403F07F067E00123244EF640159
:10241600707B900295E0FED3940840037F002290E3
:102426000296122B3A7A337986122D98EF64017050
:1024360043900296E0FE2402122B1FE0FD541EC3B9
:1024460013FF7002FF22122B09E04FF0EF700D9080
:102456000296E02402122B1FE04480F07F077E00E4
:10246600123244BF0108900295E0FF12181A123387
:102476001C7F0122900296E02402122B1FE030E01E
:0F248600037F0022900295E004F00224187F00EB
:012495002224
:102D9800EF1475F007A4900297F01202AB60282593
:102DA800E0FFE433FE900297E02402122B1FE06F4D
:102DB8007001EE60037F0022740129F9E43AFA9069
:092DC8000297E004F080D37F01C2
:012DD10022DF
:05181A00900297EFF0C1
:10181F00900183E0D394784003021938122B52FFC2
:10182F007E00123244EF7003021938122B52E490EB
:10183F000298F0900298E0FFC39406500A122B27EB
:10184F007440122B3280ECE4900298F090029BE0EF
:10185F00FEA3E0FF12324490029AEFF0602990024B
:10186F009AE025E0FF900298E0249D122B2AEFF0DA
:10187F0090029CE004F0700690029BE004F0122BA3
:10188F0033E0C3940640C57F0F7E00123244EF252C
:10189F00E044E09002A3F0900299E004F0900183FD
:1018AF00E0FF90029AF0900297E075F007A424F8F9
:1018BF00FEC3EF9E900299F0E4900298F090029987
:1018CF00E0FF900298E0C39F502290029AE0FF241D
:1018DF0002122B1FE0FE74092FF582E43401F58309
:1018EF00EEF090029AE014122B3280D1900297E022
:1018FF001475F007A490029AF0E4900298F0900209
:10190F0098E0FFC39407501A122B27E0FF90029A1A
:10191F00E02402122B1FEFF090029AE004122B32F8
:09192F0080DC900183E02407F044
:01193800228C
:0F331C0030B5FD122B46122753122B4602224EBC
:10004600EC4D6011E8497017ED33EC3304600DE4B4
:10005600FCFFFEFD22E933E8330470F80202961233
:10006600026158046009E4CC248150062850090234
:1000760002A028400302029DC0E0EB4A7044B9800A
:1000860006D0E0FB02028CEF4E701CBD8008EBFF31
:10009600EAFEE9FD80EBE98DF0A4FEE5F002012F12
:1000A600E9CDF9EAFEEBFFEF89F0A4FCE5F0CE8995
:1000B600F0A42EFFE435F0CD89F0A42DFEE435F052
:1000C6008067EF4E7005BD80D780C3EF8BF0A4AC80
:1000D600F0EE8BF0A42CFCE435F0F8EF8AF0A42CBB
:1000E600E5F038FCE433CB8DF0A42CFCE5F03BF8CE
:1000F600EE8AF0A42CFCE5F038F8E433CF89F0A4BE
:100106002CFCE5F038CF3400CE89F0A42FFFE5F0C3
:100116003EFEE433C98DF0A42EFEE5F039CD8AF01B
:10012600A42FFFE5F03EFEE43DFD33D0E0FB500793
:100136000BBB000F0202A0EC2CFCEF33FFEE33FEEC
:06014600ED33FD0202781A
:10014C000202A0EC5D046005E859047003020296FB
:10015C00120261580460F6EC4860F2EC7004FDFE8B
:10016C00FF22C860DB2481C85009C3986002500686
:10017C0002029D9850CAF582E9294B4A7005AB8260
:10018C0002028C75F0007C1A7880C3EF9BEE9AED1E
:10019C0099400DC3EF9BFFEE9AFEED99FDE842F0FE
:1001AC00DC23ACF0D0E0FFD0E0FED0E0FDAB822051
:1001BC00E7101BEB60BAEC2CFCEF33FFEE33FEEDDB
:1001CC0033FD020278E803F830E705C0F075F00063
:1001DC00EF2FFFEE33FEED33FD40B830E7C280AABF
:1001EC0075F020800E75F010800575F0087D007E8E
:1001FC00007F003392D530D50312048BEC334010C2
:10020C00EF33FFEE33FEED33FDEC33FCD5F0ED2296
:0E021C00E5F0247EA2D513CC92E7CDCEFF22D2
:10022A00EDD2E7CD33EC3392D524814006E4FFFECC
:10023A00FDFC22FCE4CFCECDCC24E0501174FF802B
:10024A00EDC3CC13CCCD13CDCE13CECF13CF0470C8
:07025A00F030D5DE02048B39
:10026100E9D2E7C933E833F892D5EDD2E7CD33ECE3
:0702710033FC5002B2D5225C
:10027800EC30E7100FBF000C0EBE00080DBD0004E7
:100288000BEB6014A2D5EB13FCED92E7FD2274FF93
:10029800FCFDFEFF22E480F8A2D574FF13FC7D80EC
:0302A800E480EF00
:030000000233D8F0
:0C33D800787FE4F6D8FD7581210231C138
:1002AB00BB010689828A83E0225002E722BBFE0251
:0902BB00E32289828A83E4932284
:1002C400BB010CE58229F582E5833AF583E02250EF
:1002D40006E92582F8E622BBFE06E92582F8E22239
:0D02E400E58229F582E5833AF583E4932253
:1002F100EF8DF0A4A8F0CF8CF0A428CE8DF0A42E21
:02030100FE22DA
:10030300BC000BBE0029EF8DF084FFADF022E4CCDE
:10031300F875F008EF2FFFEE33FEEC33FCEE9DECA7
:10032300984005FCEE9DFE0FD5F0E9E4CEFD22EDED
:10033300F8F5F0EE8420D21CFEADF075F008EF2F37
:10034300FFED33FD4007985006D5F0F222C398FD28
:050353000FD5F0EA22C5
:10035800C5F0F8A3E028F0C5F0F8E5821582700230
:060368001583E038F022CD
:10036E00E88FF0A4CC8BF0A42CFCE98EF0A42CFC2E
:10037E008AF0EDA42CFCEA8EF0A4CDA8F08BF0A4AC
:10038E002DCC3825F0FDE98FF0A42CCD35F0FCEB0B
:10039E008EF0A4FEA9F0EB8FF0A4CFC5F02ECD39D0
:0F03AE00FEE43CFCEAA42DCE35F0FDE43CFC223D
:1003BD0075F008758200EF2FFFEE33FECD33CDCCF7
:1003CD0033CCC58233C5829BED9AEC99E58298407A
:1003DD000CF582EE9BFEED9AFDEC99FC0FD5F0D657
:1003ED00E4CEFBE4CDFAE4CCF9A88222B800C1B981
:1003FD000059BA002DEC8BF084CFCECDFCE5F0CBBF
:10040D00F97818EF2FFFEE33FEED33FDEC33FCEBF7
:10041D0033FB10D703994004EB99FB0FD8E5E4F9B2
:10042D00FA227818EF2FFFEE33FEED33FDEC33FC9F
:10043D00C933C910D7059BE99A4007EC9BFCE99A93
:10044D00F90FD8E0E4C9FAE4CCFB2275F010EF2FD8
:10045D00FFEE33FEED33FDCC33CCC833C810D707D8
:10046D009BEC9AE899400AED9BFDEC9AFCE899F813
:0E047D000FD5F0DAE4CDFBE4CCFAE4C8F922A6
:102CCF00C2D5E830E70FB2D5E4C39BFBE49AFAE430
:102CDF0099F9E498F8EC30E717B2D5122D051203E5
:102CEF00F9E4C39BFBE49AFAE499F9E498F88003BA
:102CFF001203F930D50DE4C39FFFE49EFEE49DFD62
:042D0F00E49CFC2222
:0E048B00C3E49FFFE49EFEE49DFDE49CFC2282
:10049900EB9FF5F0EA9E42F0E99D42F0E89C45F0B9
:0104A9002230
:1004AA00E8600FECC313FCED13FDEE13FEEF13FF30
:0304BA00D8F12254
:1004BD00E86010ECA2E713FCED13FDEE13FEEF1355
:0404CD00FFD8F02242
:1004D100E8600FEFC333FFEE33FEED33FDEC33FC89
:0304E100D8F1222D
:0C04E400ECF0A3EDF0A3EEF0A3EFF0228B
:00000001FF
